:020000040800F2
:1040000000C0002061720008C16F0008C36F000883
:10401000C56F0008C76F0008C96F000800000000E6
:10402000000000000000000000000000CB6F00084E
:10403000CD6F000800000000CF6F0008D16F0008AE
:10404000A9720008A9720008A9720008A9720008E4
:10405000A9720008A9720008A9720008A9720008D4
:10406000A9720008A9720008A9720008D56F00089B
:10407000A9720008A9720008E16F0008ED6F00083E
:10408000F96F00080570000811700008A972000897
:10409000A9720008A9720008A9720008A972000894
:1040A000A9720008A9720008A9720008A972000884
:1040B000A9720008A9720008A9720008A972000874
:1040C000A9720008A9720008A9720008A972000864
:1040D000A97200082D70000839700008A972000844
:1040E000A9720008A9720008A9720008A972000844
:1040F000A9720008A9720008A9720008457000089A
:10410000A9720008A9720008A9720008A972000823
:1041100051700008A97200085D700008A9720008BB
:10412000A9720008A9720008A9720008A972000803
:10413000000000000000000000000000000000007F
:10414000000000000000000000000000000000006F
:10415000000000000000000000000000000000005F
:10416000000000000000000000000000000000004F
:10417000000000000000000000000000000000003F
:10418000000000000000000000000000000000002F
:10419000000000000000000000000000000000001F
:1041A000000000000000000000000000000000000F
:1041B00000000000000000000000000000000000FF
:1041C00000000000000000000000000000000000EF
:1041D00000000000000000000000000000000000DF
:0441E0005FF8E0F1B3
:1041E80010B5054C237833B9044B13B10448AFF329
:1041F80000800123237010BDDC03002000000000B4
:10420800E89D000808B5034B1BB103490348AFF309
:10421800008008BD00000000E0030020E89D0008C1
:10422800034613F8012B002AFBD1181A01387047EE
:1042380081F0004102E000BF83F0004330B54FEA4F
:1042480041044FEA430594EA050F08BF90EA020FBC
:104258001FBF54EA000C55EA020C7FEA645C7FEA4F
:10426800655C00F0E2804FEA5454D4EB5555B8BF72
:104278006D420CDD2C4480EA020281EA030382EAE3
:10428800000083EA010180EA020281EA0303362D75
:1042980088BF30BD11F0004F4FEA01314FF4801C48
:1042A8004CEA113102D0404261EB410113F0004F5A
:1042B8004FEA03334CEA133302D0524263EB430311
:1042C80094EA050F00F0A780A4F10104D5F1200EAF
:1042D8000DDB02FA0EFC22FA05F2801841F100010A
:1042E80003FA0EF2801843FA05F359410EE0A5F1DE
:1042F80020050EF1200E012A03FA0EFC28BF4CF00F
:10430800020C43FA05F3C01851EBE37101F00045C4
:1043180007D54FF0000EDCF1000C7EEB00006EEBD1
:104328000101B1F5801F1BD3B1F5001F0CD349085B
:104338005FEA30004FEA3C0C04F101044FEA4452B2
:1043480012F5800F80F09A80BCF1004F08BF5FEA39
:10435800500C50F1000041EB045141EA050130BD19
:104368005FEA4C0C404141EB010111F4801FA4F1BC
:104378000104E9D191F0000F04BF01460020B1FA11
:1043880081F308BF2033A3F10B03B3F120020CDA49
:104398000C3208DD02F1140CC2F10C0201FA0CF027
:1043A80021FA02F10CE002F11402D8BFC2F1200C8C
:1043B80001FA02F120FA0CFCDCBF41EA0C01904042
:1043C800E41AA2BF01EB0451294330BD6FEA04048B
:1043D8001F3C1CDA0C340EDC04F11404C4F1200276
:1043E80020FA04F001FA02F340EA030021FA04F388
:1043F80045EA030130BDC4F10C04C4F1200220FADF
:1044080002F001FA04F340EA0300294630BD21FA1C
:1044180004F0294630BD94F0000F83F4801306BFE2
:1044280081F480110134013D4EE77FEA645C18BFD6
:104438007FEA655C29D094EA050F08BF90EA020F6D
:1044480005D054EA000C04BF1946104630BD91EA65
:10445800030F1EBF0021002030BD5FEA545C05D168
:104468004000494128BF41F0004130BD14F58004A7
:104478003CBF01F5801130BD01F0004545F0FE411B
:1044880041F470014FF0000030BD7FEA645C1ABF50
:10449800194610467FEA655C1CBF0B46024650EA87
:1044A800013406BF52EA033591EA030F41F40021B3
:1044B80030BD00BF90F0000F04BF0021704730B539
:1044C8004FF4806404F132044FF000054FF000010E
:1044D80050E700BF90F0000F04BF0021704730B5CF
:1044E8004FF4806404F1320410F0004548BF4042A4
:1044F8004FF000013EE700BF42004FEAE2014FEAF9
:1045080031014FEA02701FBF12F07F4393F07F4FD3
:1045180081F06051704792F0000F14BF93F07F4F05
:10452800704730B54FF4607401F0004521F0004148
:1045380020E700BF50EA010208BF704730B54FF0CE
:1045480000050AE050EA010208BF704730B511F0D3
:10455800004502D5404261EB41014FF4806404F10B
:1045680032045FEA915C3FF4DCAE4FF003025FEA8D
:10457800DC0C18BF03325FEADC0C18BF033202EB15
:10458800DC02C2F1200300FA03FC20FA02F001FA6F
:1045980003FE40EA0E0021FA02F11444C1E600BF0E
:1045A80070B54FF0FF0C4CF4E06C1CEA11541DBFC1
:1045B8001CEA135594EA0C0F95EA0C0F00F0DEF88C
:1045C8002C4481EA030621EA4C5123EA4C5350EA71
:1045D800013518BF52EA033541F4801143F48013C2
:1045E80038D0A0FB02CE4FF00005E1FB02E506F053
:1045F8000042E0FB03E54FF00006E1FB03569CF0A8
:10460800000F18BF4EF0010EA4F1FF04B6F5007FAD
:1046180064F5407404D25FEA4E0E6D4146EB06061F
:1046280042EAC62141EA55514FEAC52040EA5E50A8
:104638004FEACE2EB4F1FD0C88BFBCF5E06F1ED852
:10464800BEF1004F08BF5FEA500E50F1000041EB89
:10465800045170BD06F0004646EA010140EA020036
:1046680081EA0301B4EB5C04C2BFD4EB0C0541EA58
:10467800045170BD41F480114FF0000E013C00F36D
:10468800AB8014F1360FDEBF002001F0004170BD91
:10469800C4F10004203C35DA0C341BDC04F11404AA
:1046A800C4F1200500FA05F320FA04F001FA05F236
:1046B80040EA020001F0004221F0004110EBD37003
:1046C80021FA04F642EB06015EEA430E08BF20EA2F
:1046D800D37070BDC4F10C04C4F1200500FA04F3D2
:1046E80020FA05F001FA04F240EA020001F0004164
:1046F80010EBD37041F100015EEA430E08BF20EAD7
:10470800D37070BDC4F1200500FA05F24EEA020E1E
:1047180020FA04F301FA05F243EA020321FA04F04D
:1047280001F0004121FA04F220EA020000EBD37004
:104738005EEA430E08BF20EAD37070BD94F0000F04
:104748000FD101F00046400041EB010111F4801F38
:1047580008BF013CF7D041EA060195F0000F18BFE9
:10476800704703F00046520043EB030313F4801F25
:1047780008BF013DF7D043EA0603704794EA0C0FDF
:104788000CEA135518BF95EA0C0F0CD050EA4106F5
:1047980018BF52EA4306D1D181EA030101F0004172
:1047A8004FF0000070BD50EA410606BF104619469A
:1047B80052EA430619D094EA0C0F02D150EA0136A6
:1047C80013D195EA0C0F05D152EA03361CBF1046E7
:1047D80019460AD181EA030101F0004141F0FE4186
:1047E80041F470014FF0000070BD41F0FE4141F40A
:1047F800780170BD70B54FF0FF0C4CF4E06C1CEA0A
:1048080011541DBF1CEA135594EA0C0F95EA0C0FBE
:1048180000F0A7F8A4EB050481EA030E52EA033579
:104828004FEA013100F088804FEA03334FF080559A
:1048380045EA131343EA12634FEA022245EA1115C7
:1048480045EA10654FEA00260EF000419D4208BF78
:10485800964244F1FD0404F5407402D25B084FEA25
:104868003202B61A65EB03055B084FEA32024FF4D1
:1048780080104FF4002CB6EB020E75EB030E22BF2E
:10488800B61A754640EA0C005B084FEA3202B6EBEE
:10489800020E75EB030E22BFB61A754640EA5C009D
:1048A8005B084FEA3202B6EB020E75EB030E22BF2D
:1048B800B61A754640EA9C005B084FEA3202B6EB2E
:1048C800020E75EB030E22BFB61A754640EADC00ED
:1048D80055EA060E18D04FEA051545EA16754FEA4F
:1048E80006164FEAC30343EA52734FEAC2025FEA6D
:1048F8001C1CC0D111F4801F0BD141EA00014FF0FC
:1049080000004FF0004CB6E711F4801F04BF0143CC
:104918000020B4F1FD0C88BFBCF5E06F3FF6AFAEE8
:10492800B5EB030C04BFB6EB020C5FEA500C50F178
:10493800000041EB045170BD0EF0004E4EEA1131FB
:1049480014EB5C04C2BFD4EB0C0541EA045170BD02
:1049580041F480114FF0000E013C90E645EA060E46
:104968008DE60CEA135594EA0C0F08BF95EA0C0F74
:104978003FF43BAF94EA0C0F0AD150EA01347FF4BC
:1049880034AF95EA0C0F7FF425AF104619462CE793
:1049980095EA0C0F06D152EA03353FF4FDAE1046F6
:1049A800194622E750EA410618BF52EA43067FF447
:1049B800C5AE50EA41047FF40DAF52EA43057FF4D7
:1049C800EBAE12E74FF0FF3C06E000BF4FF0010CE2
:1049D80002E000BF4FF0010C4DF804CD4FEA410C46
:1049E8007FEA6C5C4FEA430C18BF7FEA6C5C1BD013
:1049F80001B050EA410C0CBF52EA430C91EA030F94
:104A080002BF90EA020F0020704710F1000F91EAF0
:104A1800030F58BF994208BF90422CBFD8176FEABE
:104A2800E37040F0010070474FEA410C7FEA6C5C8C
:104A380002D150EA013C07D14FEA430C7FEA6C5C93
:104A4800D6D152EA033CD3D05DF8040B704700BFBF
:104A58008446104662468C461946634600E000BF0D
:104A680001B5FFF7B7FF002848BF10F1000F01BDDF
:104A78004DF808EDFFF7F4FF0CBF012000205DF8AA
:104A880008FB00BF4DF808EDFFF7EAFF34BF01202F
:104A980000205DF808FB00BF4DF808EDFFF7E0FFC8
:104AA80094BF012000205DF808FB00BF4DF808ED19
:104AB800FFF7CEFF94BF012000205DF808FB00BF80
:104AC8004DF808EDFFF7C4FF34BF012000205DF862
:104AD80008FB00BF4FEA410C7FEA6C5C02D150EA48
:104AE800013C0AD14FEA430C7FEA6C5C02D152EADE
:104AF800033C02D14FF0000070474FF001007047AF
:104B08004FEA410212F5001215D211D56FF47873ED
:104B1800B3EB625212D94FEAC12343F0004343EA90
:104B2800505311F0004F23FA02F018BF404270476B
:104B38004FF00000704750EA013005D111F00040F5
:104B480008BF6FF0004070474FF00000704700BF8B
:104B580038B50E4B054618784FF47A73B3FBF0F36B
:104B68000B4A1068B0FBF3F000F04CFB044658B950
:104B78000F2D09D8024629464FF0FF3000F000FB00
:104B8800044B20461D6038BD012038BD00000020C0
:104B98000802002004000020074A08B51368032013
:104BA80043F01003136000F0D9FA0020FFF7D0FF9C
:104BB80002F05CF8002008BD00200240034A044BC4
:104BC80011681B780B441360704700BF2004002055
:104BD80000000020014B1868704700BF2004002027
:104BE80038B50446FFF7F6FF0546631C1EBF044BA5
:104BF8001B78E418FFF7EEFF401B8442FAD838BD53
:104C0800000000207047436A10B59A6A12F0500FEE
:104C18001BD19A6A42F400729A621A68926802F486
:104C28006022B2F5602F0CD11A7B52B99A6A22F42D
:104C380080729A629A6AD2045EBF9A6A42F001024E
:104C48009A621846FFF7DEFF10BD1B6ABDE81040E8
:104C58001B6B1847704708B5406AFFF7FBFF08BD94
:104C68007047036810B55A680446900627D51A6835
:104C7800910724D5A26AD2065EBFA26A42F40072E6
:104C8800A2629A6802F46022B2F5602F10D1227BEA
:104C980072B95A6822F020025A60A36A23F480731A
:104CA800A362A36ADB045EBFA36A43F00103A362A5
:104CB8002046FFF7A7FF6FF0120223681A602368E7
:104CC8005A68100630D51A6851072DD5A26AD2063F
:104CD8005EBFA26A42F40052A2629A6802F4E042FD
:104CE800B2F5E04F0AD05A68500516D49A6802F413
:104CF8006022B2F5602F10D1227B72B95A6822F077
:104D080080025A60A36A23F48053A362A36AD90578
:104D18005EBFA36A43F00103A362204600F01CFAB9
:104D28006FF00C0223681A6023685A6852060DD582
:104D38001B68DB070AD5A36A204643F48033A362C5
:104D4800FFF78EFF6FF0010223681A6010BD7047ED
:104D5800406A08B5836A43F040038362C36A43F03C
:104D68000403C362FFF7F3FF08BD0000002373B517
:104D7800019390F82430012B74D001234D6880F8FA
:104D88002430062D02684FEA85030C6825D82B4489
:104D98001F25566B053B9D4026EA050504FA03F3DB
:104DA8002B435363092C4FEA44038D682FD90726F8
:104DB8002344D1681E3B9E4021EA060105FA03F30D
:104DC8000B43D360A4F11003012B2BD9002300223D
:104DD80080F82420184602B070BD0C2D0BD82B4447
:104DE8001F25166B233B9D4026EA050504FA03F3AD
:104DF8002B431363D6E72B441F25D66A413B9D40BE
:104E080026EA050504FA03F32B43D362CAE707260B
:104E1800116923449E4021EA060105FA03F30B4376
:104E28001361CFE7104B9A4216D193681B02CDD479
:104E38009368102C43F400039360C7D10B4B0C4AC2
:104E48001B68B3FBF2F20A2353430193019B002B27
:104E5800BCD0019B013BF8E7836A43F020038362DF
:104E68000123B4E70223B5E700240140080200202B
:104E780040420F00002373B50193036804469A6803
:104E8800D20702D5002002B070BD9A6842F0010234
:104E98009A60124B124A1B68B3FBF2F30193019B11
:104EA800C3B9FFF797FE064623689D6815F001050C
:104EB800E8D1FFF78FFE801B0228F5D9A36A84F892
:104EC800245043F01003A362E36A012043F0010376
:104ED800E362D8E7019B013BE0E700BF080200203E
:104EE80040420F002DE9D8419046404B02680446E5
:104EF8009A420F4602D03E498A4203D15B6813F4B6
:104F0800702F6ED194F82430012B6CD001232046E9
:104F180084F82430FFF7AEFF064600285DD1A06A6A
:104F2800216820F47060324B20F0010040F480705A
:104F38009942A06204D12D4A536813F4702F3ED1D0
:104F4800A36A23F48013A3624B685A0505D5A36AA4
:104F580023F4405343F48053A362A36A206A13F4F2
:104F6800805318BFE36A3A4618BF23F00603E3628A
:104F7800002384F824301F4B4C3183621E4BC362DC
:104F88001E4B03636FF0020341F84C3C51F8443C5C
:104F980043F4807341F8443C434600F089F92368A0
:104FA8009A6802F46022B2F5602F9A680CBF42F446
:104FB800A00242F480129A603046BDE8D881A36A04
:104FC80043F48013A36253685B0541BFA06A20F4D1
:104FD800405040F48050A062BFE7002384F824309A
:104FE800EAE70126E8E70226E6E700BF00240140D9
:104FF800002801400F4C00085F4C0008594D00087C
:1050080038B5036804469A68D20701D4002038BD31
:105018009A6822F001029A60FFF7DCFD05462368D2
:105028009B68DB07F2D5FFF7D5FD401B0228F6D9B0
:10503800A36A012043F01003A362E36A43F001036B
:10504800E36238BDF8B50446002877D0836A23B9EF
:10505800C36280F8243001F02BFE2046FFF7D0FF12
:10506800A36A13F010036BD1002869D1A26A3749EB
:1050780022F4885222F0020242F00202A26294E86C
:1050880024008A42E16904D1B1F5402F08BF4FF4EA
:105098000021267B45EA46052943A568B5F5807FAA
:1050A80035D0012D08BF4FF48073277D012F06D11D
:1050B8007EBBA669013E43EA463343F40063566863
:1050C800B5F5807F26F4694643EA0603536096687F
:1050D8001F4B03EA060343EA0103936001D0012D45
:1050E80020D12369013B1B05D56A25F470052B43A4
:1050F800D3629268174B1340994215D10023E3629B
:10510800A36A23F0030343F00103A362F8BD2B460F
:10511800CBE7A66A46F02006A662E66A46F00106D4
:10512800E662CCE70023DFE7A36A23F0120343F02B
:105138001003A362E36A43F00103E3620120F8BDB0
:10514800A36A43F01003A362F8E700BF003C0140E4
:10515800FDF7E1FFFE0E1FFF70470000074A00023F
:10516800D36800F4E06023F4E0631B041B0C43F0F5
:10517800BF6343F400330343D360704700ED00E09E
:10518800174B30B5DC68C4F30224C4F10703251DAE
:10519800042B28BF0423062D4FF0010598BF0024D7
:1051A80005FA03F303F1FF3388BF033C1940A1401C
:1051B80005FA04F4013C2240002842EA01024FEAC1
:1051C8000212A9BF00F16040064BD2B200F561405F
:1051D800BBBF00F00F00D2B280F800231A5430BDD4
:1051E80000ED00E014ED00E0002808DB012342098F
:1051F80000F01F0003FA00F0014B43F8220070474B
:1052080000E100E00138B0F1807F0AD2F021064BBE
:10521800064A586082F823100020072298601A6016
:1052280070470120704700BF10E000E000ED00E08B
:1052380010B5002832D00168194B1424994225D89A
:10524800184AA3F207430A44B2FBF4F2920002643C
:105258008468C36343680A682343C46822F47F529E
:105268002343046922F030022343446923438469B9
:105278002343C469234313430B600122002380F8AE
:105288002120836380F82030184610BD064B0B445C
:10529800B3FBF4F39B000364044BD9E7012010BD72
:1052A80007040240F8FFFDBFF8FBFDBF0004024001
:1052B800F0B590F82040012C35D0012490F8215009
:1052C80080F82040A5424FF000064FF0020428D194
:1052D80080F82140046886632668076C26F001067A
:1052E8002660C66BBD407560636043680568102B17
:1052F800C36A0BBFA260A160E160E2604BB12368A2
:1053080043F00E0323602B68002043F001032B6059
:10531800F0BD236823F004032360236843F00A03E5
:10532800F0E780F820600220F0BD000090F82130FE
:1053380010B5022B03D004238363012010BD03683A
:105348001A6822F00E021A601A6822F001021A6026
:10535800294A934224D902F56272934219D0143231
:10536800934218D01432934217D0143293420CBF90
:105378004FF480534FF48033204A536001230024B4
:1053880080F82130436B80F820409BB39847204633
:1053980010BD0123F0E71023EEE74FF48073EBE72D
:1053A80017498B4216D014318B4215D014318B42D9
:1053B80014D014318B4214D014318B4214D01431D0
:1053C8008B4214D0934214BF4FF480334FF0807354
:1053D8000C4AD2E70123FBE71023F9E74FF4807367
:1053E800F6E74FF48053F3E74FF48033F0E74FF4D8
:1053F8008013EDE7184610BD80000240000402400B
:10540800080002400000024070B40425C66B026C1C
:105418003468036895402542196855D04D0753D51F
:105428001A6896065EBF1A6822F004021A60604A7B
:1054380093421FD902F56272934214D014329342F8
:1054480013D01432934212D0143293420CBF4FF44B
:1054580080434FF48023574A5360C36A002B00F0FF
:10546800A58070BC18470423F5E74023F3E74FF401
:105478008063F0E750498B4216D014318B4215D027
:1054880014318B4214D014318B4214D014318B4216
:1054980014D014318B4214D0934214BF4FF480239C
:1054A8004FF08063454AD7E70423FBE74023F9E739
:1054B8004FF48063F6E74FF48043F3E74FF480231B
:1054C800F0E74FF48003EDE702259540254257D0D9
:1054D8008D0755D51A68940606D41A6822F00A0270
:1054E8001A60012280F82120314A93421ED902F520
:1054F8006272934213D01432934212D01432934200
:1055080011D0143293420CBF4FF400534FF40033C0
:10551800284A5360002380F82030836A9EE70223DC
:10552800F6E72023F4E74FF40073F1E722498B42B2
:1055380016D014318B4215D014318B4214D014314B
:105548008B4214D014318B4214D014318B4214D0B6
:10555800934214BF4FF400334FF00073174AD8E753
:105568000223FBE72023F9E74FF40073F6E74FF433
:105578000053F3E74FF40033F0E74FF40013EDE77F
:1055880008259540254211D009070FD5196821F043
:105598000E011960012303FA02F27260836380F836
:1055A8002130002380F82030036B57E770BC704728
:1055B800800002400004024008000240000002404F
:1055C8002DE9F74F002426466C4F6D4BDFF8B8E104
:1055D800DFF8B8C10A6832FA06F502D103B0BDE8AF
:1055E800F08F4FF0010808FA06F802EA0802904521
:1055F80040F084804D68122D00F0B18000F2878061
:10560800022D00F0A9807BD8002D00F08C80012DA0
:1056180000F0A0804FF00F09FF2A93BF824606F1E1
:105628008045083DD0F800B092BFB500D0F804B06E
:10563800AD0009FA05F82BEA080804FA05F588BF51
:1056480000F1040A48EA0505CAF80050D1F804A098
:105658001AF0805F52D0BD6926F0030845F00105B5
:10566800BD61BD6908F1804805F00105019508F59F
:10567800803806F0030B019D4FEA8B0BD8F80850D1
:1056880009FA0BF925EA09093E4DA8426CD005F53F
:105698008065A8426AD005F58065A84268D005F5FE
:1056A8008065A84266D005F58065A84264D070453B
:1056B8000CBF0525062505FA0BF545EA0905C8F8C6
:1056C80008501D681AF4803F14BF154395431D60A8
:1056D8005D681AF4003F14BF154395435D609D68EB
:1056E8001AF4801F14BF154395439D60DD681AF4B2
:1056F800001F14BF2A4325EA0202DA60013669E76F
:10570800032D25D0112D85D1CC68043482E7654559
:1057180009D012D8DFF878904D4504D009F58039C2
:105728004D457FF477AF8C68E4B1012C0CBFC0F80D
:105738001080C0F8148008246CE7DFF858904D45B5
:10574800F1D009F580394D45EDD0A9F58019E7E785
:1057580000245FE7CC685DE7CC6808345AE7CC687A
:105768000C3457E7042455E70025A4E70125A2E7F0
:105778000225A0E703259EE704259CE700100240C8
:105788000004014000080140001C014000002110F5
:1057980000001110000031100AB1016170470904BE
:1057A800FBE7C3680B4214BF416101617047000009
:1057B8002DE9F341054608B901203CE00368DB0701
:1057C80010D42B689F075DD42B68190700F19480CB
:1057D8002B685A0700F1BE80E869002840F02C8148
:1057E800002028E08F4C636803F00C03042B07D0DB
:1057F800636803F00C03082B09D16368DE0306D540
:1058080023689C03DDD56B68002BDAD1D4E76B687D
:10581800B3F5803F12D1236843F480332360FFF748
:10582800D9F9064623689803CBD4FFF7D3F9801B30
:105838006428F7D9032002B0BDE8F0819BB923683A
:1058480023F480332360236823F480232360FFF745
:10585800C1F9064623689903B3D5FFF7BBF9801B46
:105868006428F7D9E6E7B3F5A02F236803D143F4FA
:1058780080232360CFE723F480332360236823F455
:105888008023CBE7674C636813F00C0F07D063687D
:1058980003F00C03082B10D16368DA030DD42368D6
:1058A8009B0702D52B69012B86D123686A6923F0EF
:1058B800F80343EAC203236086E72A695A4B6AB1B0
:1058C80001221A60FFF786F9064623689F07ECD481
:1058D800FFF780F9801B0228F7D9ABE71A60FFF7BA
:1058E80079F90646236898077FF56EAFFFF772F9D6
:1058F800801B0228F6D99DE7AA694A4C4B4BDAB1BE
:1059080001221A60FFF766F90646636A9B070DD500
:105918004FF4FA52464B1B68B3FBF2F3019300BFF6
:10592800019B5A1E0192002BF9D151E7FFF752F95A
:10593800801B0228E9D97DE71A60FFF74BF9064674
:10594800636A9F077FF544AFFFF744F9801B02287D
:10595800F6D96FE7334CE369D80024D40127E3690B
:1059680043F08053E361E36903F080530093009BA5
:10597800304E3368D90518D5EB68012B26D1236A38
:1059880043F001032362FFF725F941F28836804688
:10599800236A9B073FD5002F3FF41EAFE36923F02E
:1059A8008053E36118E70027E2E7336843F4807324
:1059B8003360FFF70FF980463368DA05DCD4FFF768
:1059C80009F9A0EB08006428F6D933E7ABB9236AD4
:1059D80041F2883823F001032362236A23F0040389
:1059E8002362FFF7F7F80646236A9807D3D5FFF72F
:1059F800F1F8801B4045F7D91CE7052B236A03D132
:105A080043F004032362BAE723F001032362236A05
:105A180023F00403B6E7FFF7DDF8A0EB0800B04277
:105A2800B6D907E700100240000042428004424213
:105A380008020020007000402A4B5A681C4602F0F9
:105A48000C02082A3DD00023274E022833602BD1B0
:105A5800FFF7C0F80746236899011FD42B6AB3F5EE
:105A6800803F05D16268A96822F400320A43626067
:105A7800696A62680B4322F474121343636001235A
:105A88003360FFF7A7F8054623689A013FF5A8AEEB
:105A9800FFF7A0F8401B0228F6D9CBE6FFF79AF8E3
:105AA800C01B0228D7D9C5E6FFF794F80546236836
:105AB8009B017FF595AEFFF78DF8401B0228F6D9BC
:105AC800B8E601283FF4B7AE58682B6A00F4803274
:105AD8009A427FF471AE6B6A00F47010C01A18BF56
:105AE8000120A8E6001002406000424230B5194B80
:105AF80087B002AC03F110052246186859680833CC
:105B080003C2AB421446F7D101238DF804300223B7
:105B180011498DF805304B6803F00C02082A17D19B
:105B2800C3F3834206A80244DB0312F8102C0CD5F9
:105B38004B680A48C3F34043504306AA134413F87A
:105B4800143CB0FBF3F007B030BD05485043FAE70A
:105B58000248F8E7009E00080010024000127A0090
:105B680000093D002DE9F0410D46044610B9012019
:105B7800BDE8F081454A136803F007038B4229D337
:105B880021688E0731D4CA0744D4404A136803F009
:105B980007039D4267D322683D4D12F0040F6ED172
:105BA800130706D56B68226923F4605343EAC203DE
:105BB8006B60FFF79BFF6B68364AC3F30313D35C34
:105BC800D840354B1860354B1868FEF7C1FF0020E8
:105BD800BDE8F081136823F007030B4313601368D3
:105BE80003F007039942C2D1CAE7294B11F0040F09
:105BF8001EBF5A6842F4E0625A60080742BF5A68FA
:105C080042F460525A605A68A06822F0F0020243D7
:105C18005A60B8E762681E4E012A33681BD113F434
:105C2800003FA4D0736841F2883823F0030313437C
:105C38007360FEF7CFFF07467368626803F00C03D2
:105C4800B3EB820FA1D0FEF7C5FFC01B4045F3D9C7
:105C58000320BDE8F081022A02D113F0007FE0E7BB
:105C680013F0020FDDE7136823F007032B431360DB
:105C7800136803F007039D427FF479AF8BE76B68E5
:105C8800E16823F4E0630B436B6089E7002002407E
:105C980000100240DC9E00080802002004000020DA
:105CA800044B054A5B68C3F30223D35C034A1068BC
:105CB800D840704700100240EC9E000808020020FF
:105CC800044B054A5B68C3F3C223D35C034A1068DC
:105CD800D840704700100240EC9E000808020020DF
:105CE80003682DE9F341D907054620D5354CE3690A
:105CF800DA0032D40127E36943F08053E361E369B2
:105D080003F080530193019B2F4E3368DB0526D5A2
:105D1800236A13F4407336D1236A6A6823F4407304
:105D2800134323621FB1E36923F08053E3612868BA
:105D3800830706D5234AA968536823F440430B43D5
:105D4800536010F010001BD01E4A69695368002088
:105D580023F480030B43536012E00027D4E7336831
:105D680043F480733360FEF735FF80463368D80507
:105D7800CED4FEF72FFFA0EB08006428F6D9032045
:105D880002B0BDE8F0816A6802F440729342C3D061
:105D980001200E4A236A1060002023F4407110602D
:105DA8002162D907B8D5FEF715FF41F288380646B3
:105DB800236A9A07B0D4FEF70DFF801B4045F7D938
:105DC800DDE700BF0010024000700040400442427E
:105DD80003680020DA6842F00102DA609A6802F08B
:105DE8000702062A1EBF1A6842F001021A607047AD
:105DF8007047704770477047036810B51A690446C2
:105E080091070ED5DA6892070BD56FF002021A6176
:105E180001229B6902779B0777D0FFF7EAFF0023EF
:105E2800237723681A69500710D5DA6851070DD50A
:105E38006FF004021A6102229B69227713F4407FF3
:105E4800204668D0FFF7D5FF0023237723681A6917
:105E580012070FD5DA6810070CD56FF008021A611F
:105E68000422DB692277990720465AD0FFF7C1FF41
:105E78000023237723681A69D20610D5DA68D0067A
:105E88000DD56FF010021A610822DB69227713F42E
:105E9800407F20464BD0FFF7ACFF002323772368D1
:105EA8001A69D10708D5DA68D20705D56FF001025B
:105EB80020461A6100F058FC23681A69100608D5B4
:105EC800DA68110605D56FF0800220461A6100F0E5
:105ED800BAF823681A69520608D5DA68500605D553
:105EE8006FF0400220461A61FFF785FF23681A69A0
:105EF800910622D5DA6892061FD56FF02002204657
:105F0800BDE810401A6100F09DB8FFF771FF204608
:105F1800FFF770FF83E7FFF76BFF2046FFF76AFF85
:105F280092E7FFF765FF2046FFF764FFA0E7FFF75A
:105F38005FFF2046FFF75EFFAFE710BD244A036806
:105F4800904212D002F5006290420ED0B0F1804F1C
:105F58000BD0A2F59832904207D002F580629042A9
:105F680003D002F5806290421DD14A6823F0700385
:105F78001343174A904212D002F5006290420ED0A5
:105F8800B0F1804F0BD0A2F59832904207D002F5BD
:105F98008062904203D002F58062904203D1CA68C1
:105FA80023F4407313434A6923F0800313430360C7
:105FB8008B68C3620B688362054B984203D003F574
:105FC8000063984201D10B69036301234361704761
:105FD800002C014010B50446A0B190F83D3003F004
:105FE800FF021BB980F83C2000F0ECFE0223206879
:105FF80084F83D30211DFFF7A1FF0123002084F81C
:106008003D3010BD012010BD90F83C3030B5012B5B
:106018004FF0020314D0046880F83D306268A3682A
:106028000D68496822F0700223F080030B432A436D
:106038006260A360012380F83D30002380F83C3083
:10604800184630BD704770470368DA6822F49072CA
:10605800DA605A6922F001025A61202380F83A3046
:106068007047000038B505460368C1681A691924E5
:1060780022F440520A431A6182680069D9680243CF
:10608800686921F4B05121F00C0102430A43DA6037
:106098005A69A96922F440720A435A610D4A934227
:1060A80014D1FFF70DFE60436C686422A400B0FBB6
:1060B800F4F0B0FBF2F402FB14031B013233B3FB20
:1060C800F2F3296803EB04138B6038BDFFF7E8FD92
:1060D800E9E700BF00380140F8B504460E46174608
:1060E8001D4621680B6836EA030301D10020F8BD7C
:1060F8006B1CF7D095B923680320DA6822F4D072B4
:10610800DA605A6922F001025A61202384F8393092
:1061180084F83A30002384F83830F8BDFEF75AFD89
:10612800C01B8542DDD2E6E710B5044640B390F8BF
:10613800393003F0FF021BB980F8382000F056FE12
:106148002423226884F83930D368204623F4005386
:10615800D360FFF787FF236800201A6922F4904272
:106168001A615A6922F02A025A61DA6842F4005226
:10617800DA602023E06384F8393084F83A3010BDBF
:10618800012010BD2DE9F0411F4690F83930044632
:10619800202B0D4690464ED1002949D0002A47D0E1
:1061A80090F83830012B46D0012380F8383000238E
:1061B800C363212380F83930FEF70CFD0646A4F8A6
:1061C8002480A4F82680E38C9BB26BB93B46324608
:1061D80040212046FFF780FFA8B9202384F8380023
:1061E80084F83930BDE8F081E38C3246013B9BB23C
:1061F800E384A3688021B3F5805F20463B460ED137
:10620800FFF76AFF10B10320BDE8F0812B882268F0
:10621800C3F308035360236943B90235D3E7FFF793
:106228005BFF0028EFD123682A785A600135CAE756
:106238000120BDE8F0810220BDE8F08138B50446B0
:10624800134694F83920202A2AD139B333B394F865
:106258003820012A24D00122002584F83820212260
:10626800E384206BE56384F839200E4AA384216215
:1062780082620D4A4563C2620C4A02632268043294
:10628800FFF716F86FF04002236828461A605A692B
:1062980084F8385042F080025A6138BD012038BD78
:1062A800022038BD4B630008796300084564000884
:1062B800134690F83A2073B5202A054638D10029AC
:1062C80034D0002B32D090F83820012A30D0012267
:1062D800002480F83820222281628385C46380F8F4
:1062E8003A20406B134A2E688262134A4463C262A2
:1062F800124A02630A46311DFEF7DAFF20462B6870
:1063080001941A6801925A6885F838400192019AF6
:10631800DA6842F48072DA605A6942F001025A611E
:106328005A6942F040025A6102B070BD0120FBE791
:106338000220F9E78363000839640008456400080F
:10634800704708B50368426A1B6813F020030AD136
:10635800D38413685A6922F080025A61DA6842F0DD
:106368004002DA6008BD1046FFF7EAFF08BD704733
:1063780008B5406AFFF7FBFF08BD08B50368426A25
:106388001B6813F0200310D1D3851368D96821F452
:106398008071D960596921F001015961596921F069
:1063A80040015961202382F83A30104600F018FF66
:1063B80008BD90F83A3010B5222B36D183680169B0
:1063C800B3F5805F0268836A23D15268E9B9C2F3E2
:1063D800080223F8022B8362C48D013CA4B2C48551
:1063E8008CB90368DA6822F02002DA60DA6822F4ED
:1063F8008072DA605A6922F001025A61202380F81B
:106408003A3000F0EDFE002010BDD2B223F8012B87
:10641800E1E721B9591C526881621A70DCE75268B9
:10642800591C816202F07F02F7E7022010BD704715
:1064380008B5406AFFF7FBFF08BD7047416A08B519
:106448000B685A6991F8390021280AD1120608D533
:106458000022CA84DA6822F0C002DA60202281F8B9
:1064680039205B6991F83A20222A06D15B0604D5C7
:1064780000230846CB85FFF7E7FDCB6B084643F0C2
:106488001003CB63FFF7D9FF08BD0000036870B5A0
:106498001A6804461607D9685D6907D196065AD561
:1064A8008D0658D5BDE87040FFF783BF15F001058C
:1064B80002D111F4907F4ED0D30705D5CE0542BF47
:1064C800E36B43F00103E363500704D51DB1E36BAD
:1064D80043F00203E363930704D51DB1E36B43F074
:1064E8000403E363160704D51DB1E36B43F0080307
:1064F800E363E36B002B66D0950604D5880602D5C6
:106508002046FFF756FF236820465D69E26B1107B6
:1065180002D415F040051AD0FFF796FD23685A6992
:10652800520610D55A69606B22F040025A6150B188
:10653800254B4363FEF7FAFE002844D0606BBDE8A4
:106548007040436B18472046FFF777FF70BDFFF791
:1065580074FFE56370BD160627D50D0625D594F89A
:106568003920212A2FD1A268B2F5805F226A17D17B
:106578001188C1F308015960216979B90232226290
:10658800E28C013A92B2E284EAB9DA6822F0800237
:10659800DA60DA6842F04002DA6070BD0132EEE794
:1065A800511C216212785A60EAE750060BD54A0658
:1065B80009D5DA68204622F04002DA60202384F800
:1065C8003930FFF7BDFE70BDD565000808B500235A
:1065D800406AC385C384FFF730FF08BD002310B5A8
:1065E8000F4CC90007290FDC61B141F2210213F4F5
:1065F800004F4FEA43039BB201F1FF3118BF5340EC
:106608000029F4D1184610BD10F8012B083982EA88
:10661800132234F8122082EA03239BB2E2E700BF78
:1066280008000020174B10B51A78174C12B12278C1
:10663800032A10D801221A702378032B0BD8DFE81D
:1066480003F0020B0E110D21104800F0FDFD237818
:106658000133DBB2237010BD0D210D48F5E71D2174
:106668000C48F2E715210C4800F0EEFD0520FEF776
:10667800B7FA0A21094800F0E7FD094801F032FBA2
:10668800E5E700BFF8030020F90300201B9E00087F
:10669800299E0008379E0008559E00086B9E00083A
:1066A800769E000838B504460D46FDF7B9FD00236F
:1066B800C0B2834201DB002038BDE15C2A789142F8
:1066C80001D1D8B238BD0133F3E70000F7B520494E
:1066D80001F0C6FB00231E49064600938DF80430DE
:1066E80001F0BEFB88B31B493046FFF7DBFF0446C9
:1066F80010B333185A78BE2A1ED113F8022C13F897
:10670800013C68468DF801308DF8002000F0C9FD85
:1067180005463046FDF784FDC1B20F4801F05AFA2C
:10672800631CECB21C440D4DF7180834BB1B9C428B
:1067380005DA0B4801F0D6FA002003B0F0BD17F8CF
:10674800011B284601F046FAF0E70648F2E700BFC9
:106758008D9E0008969E0008989E0008A89E000836
:106768008B9E0008AC9E000802680A4B9A420FD123
:10677800094A136801331360084A13680133136028
:10678800074A136801331360064A1368013313601C
:10679800704700BF001000400804002004040020D7
:1067A80000040020FC03002010B514460A23024808
:1067B800FFF7E8FC204610BDFC05002010B596B098
:1067C800282200210CA800F09BFD1422002101A81A
:1067D80000F096FD182200210DEB020000F090FD5C
:1067E800012310931023022411934FF460130CA873
:1067F80015930C941394FEF7DBFF0F234FF480627C
:1068080001930023214601A803930492059302945F
:10681800FFF7A8F94FF4004306A806940893FFF77A
:106828005FFA16B010BD00002DE9F04FBE4A8FB0D8
:106838005168106807AB03C31189927ABB4D198060
:106848009A70FEF7A9F9FFF7B9FF102200210AA8EC
:1068580000F056FDAB69002243F01003AB61AB6951
:1068680049F2400103F010030393039BAB69B0485E
:1068780043F00403AB61AB69002403F00403049301
:10688800049BAB69012643F00803AB61AB6902279F
:1068980003F008030593059BAB694FF4602843F0A8
:1068A8002003AB61AB694FF0090B03F0200306939B
:1068B800069BFEF771FF00224EF2F2019D48FEF79B
:1068C8006BFF002248F2D8019B48FEF765FF0022C3
:1068D80004219A48FEF760FF49F240030AA9944848
:1068E8000A930B960C940D97FEF76AFE4EF2F2038C
:1068F8000AA990480A930B960C940D97FEF760FE30
:1069080048F2D8030AA98C480A930B960C940D9761
:10691800FEF756FE04230AA988480A930B960C949E
:106928000D97FEF74DFE6B69854F33436B616B69BD
:10693800844D33400293029B834B28460A940B9460
:106948000C942B60AC602E732C75C5F81C806C60A1
:106958002E61FEF777FB07230AA92846CDF828B051
:106968000B960C93FEF702FA784B38463B60BC60F6
:106978003C733C75C7F81C807C603E610A940B949C
:106988000C94FEF75FFB0A234FF00B090AA938465F
:106998006F4F0A930B960C94FEF7E8F96D4B384647
:1069A8003B60BC603C733C75C7F81C807C603E61F2
:1069B8000A940B940C94FEF745FB0AA938460B96EB
:1069C8000C94CDF82890FEF7D1F941F6FF03DFF8D3
:1069D800A4A1614A50468AE80C000A940B94CAF8AC
:1069E8000840CAF80CB0CAF81840FFF7F3FA0AA929
:1069F8005046DFF884810A940B94FFF705FB574B48
:106A08004FF00C0BC8F800304FF4E133544F4046B8
:106A1800C8F804300193C8F80840C8F80C40C8F812
:106A28001040C8F81840C8F81C40C8F814B0FFF760
:106A38007BFB4C4A019B38463A607B60BC60FC603B
:106A48003C61BC61FC61C7F814B0FFF76DFB019BAA
:106A58004548464A436002608460C46004618461BA
:106A6800C461C0F814B0FFF75FFB2246214610202E
:106A7800FEF786FB1020FEF7B7FB224621460F20C3
:106A8800FEF77EFB0F20FEF7AFFB224621460E20C5
:106A9800FEF776FB0E20FEF7A7FB224621461120C3
:106AA800FEF76EFB1120FEF79FFB224621462F20A2
:106AB800FEF766FB2F20FEF797FB2246214634207F
:106AC800FEF75EFB3420FEF78FFB22462146362078
:106AD800FEF756FB3620FEF787FB2246214612209A
:106AE800FEF74EFB1220FEF77FFB224621462520AB
:106AF800FEF746FB2520FEF777FB22462146262097
:106B0800FEF73EFB2620FEF76FFB2246214648464D
:106B1800FEF736FB4846FEF767FB5046FFF758F985
:106B2800134B21461B6829E0109E00080010024004
:106B38000010014000080140000C01400014014011
:106B4800A004002014050020002401400028014072
:106B580044050020003C014000100040003801407E
:106B68000007002000440040C0060020004C004000
:106B78000C02002080060020FC0500202E4C98689E
:106B880001F0B8F82D4801F0ADF8494607A8FFF71D
:106B980025FD01462A4801F01DF82A49404600F023
:106BA800B9FA3846284900F0B5FA32462749284646
:106BB800FEF798F92646264F264D2B68B3F5FA7F3F
:106BC80005D902213846FEF7ECFD00232B60224D43
:106BD8002B68B3F57A7F03D9FFF724FD00232B60D8
:106BE80040F6B8321D4B1968914284BF00221A60E2
:106BF8002368B3F5967F02D900F0AAFAA0B901205C
:106C0800FDF7EEFFD8E7404600F0A8FAAB68002B86
:106C1800F9DC0D4DDFF84880AB68002B08DC00205C
:106C2800306000F08FFAEAE7064DDFF83880EDE7CC
:106C3800404600F093FAEFE708040020BC9E0008E5
:106C4800C99E0008440B0020500F00202404002097
:106C5800000801400404002000040020FC03002078
:106C680000070020FC050020704700000E4B82B092
:106C78009A6942F001029A619A6902F0010200924F
:106C8800009ADA6942F08052DA61DB69074A03F058
:106C980080530193019B536823F0E06343F08063C2
:106CA800536002B0704700BF00100240000001406E
:106CB80030B505468BB01022002106A800F020FB55
:106CC8002B68384A934235D1374B38489A6906A918
:106CD80042F400729A619A69354C02F4007200928B
:106CE800009A9A6942F008029A619B6903F00803C6
:106CF8000193019B0223069303230793FEF760FC8D
:106D08008022E2604FF4007222614FF40062294B46
:106D1800626123602022002320466360A360A26191
:106D2800E361FEF785FA08B1FFF79EFF2C62656202
:106D38000BB030BD204A93421BD11B4B9A6942F4D9
:106D480080629A619A6902F480620292029A9A6950
:106D580042F010029A619B6903F010030393039BAE
:106D680001230693032306A914480793FEF728FC7A
:106D7800DEE7134A9342DBD10B4B9A6942F4004297
:106D88009A619A6902F400420492049A9A6942F05C
:106D980010029A619B6903F010030593059B022377
:106DA800DFE700BF0024014000100240000C014052
:106DB8003C06002008000240002801400010014065
:106DC800003C01400268084B82B09A420AD103F5A0
:106DD8000033DA6942F01002DA61DB6903F010036C
:106DE8000193019B02B070470010004070B5054642
:106DF8008AB01022002106A800F082FA2B68604AA7
:106E0800934229D15F4B06A9DA695F4842F4002210
:106E1800DA61DA6902F400220092009A9A6942F073
:106E280010029A619B6903F010030193019B4FF4D0
:106E3800806306930223079303230993FEF7C0FB9D
:106E48004FF400630693002306A94F48079308935D
:106E5800FEF7B6FB0AB070BD4C4A934250D1494B7D
:106E680006A99A694A4842F480429A619A690026BA
:106E780002F480420292029A9A69464C42F0040255
:106E88009A619B6903F004030393039B4FF4007317
:106E980006930223079303230993FEF791FB4FF40C
:106EA80080633B4806A9069307960896FEF788FB79
:106EB800394B204684E848008023A660E3602661B9
:106EC8006661A661E661FEF7B3F908B1FFF7CCFE8B
:106ED8006C636562314B324C2360102380226360FF
:106EE8000023E260A36023616361A361E36120463C
:106EF800FEF79EF908B1FFF7B7FE2C636562A9E7B4
:106F0800284A9342A6D11F4B06A9DA69204842F4C1
:106F18000032DA61DA69002602F400320492049A37
:106F28009A69214C42F004029A619B6903F00403B8
:106F38000593059B042306930223079303230993D0
:106F4800FEF73EFB0823124806A906930796089603
:106F5800FEF736FB154B204684E848008023A660E0
:106F6800E36026616661A661E661FEF761F908B132
:106F7800FFF77AFE6C6365620D4B0E4CACE700BF01
:106F8800004C004000100240001001400038014051
:106F980000080140740500205800024044000240E7
:106FA800D0040020004400405C0400206C00024033
:106FB80080000240B80500207047FEE7FEE7FEE7C4
:106FC800FEE7704770477047FDF7F8BD0148FEF7C8
:106FD8001BBA00BF3C0600200148FEF715BA00BFE7
:106FE800D00400200148FEF70FBA00BF7405002046
:106FF8000148FEF709BA00BF5C0400200148FEF70B
:1070080003BA00BFB805002008B50448FDF729FEFB
:10701800BDE808400248FDF724BE00BF1405002063
:10702800A00400200148FFF731BA00BFFC0500208A
:107038000148FFF72BBA00BF000700200148FDF701
:1070480010BE00BF440500200148FFF71FBA00BF6B
:10705800C00600200148FEF7CFBE00BF8006002012
:1070680070B50E4615460C46A31B9D4201DC28460A
:1070780070BDAFF3008004F8010BF5E708B50A4BC3
:107088000246196809B9094919606946186802442D
:107098008A4206D900F00AF90C2303604FF0FF304A
:1070A80008BD1A6008BD00BF0C0400206013002052
:1070B8004FF0FF3070474FF4005300204B6070478B
:1070C80001207047002070470E4B1A6842F00102F9
:1070D8001A6059680C4A0A405A601A6822F0847289
:1070E80022F480321A601A6822F480221A605A68E0
:1070F80022F4FE025A604FF41F029A60034A044BBE
:107108009A607047001002400000FFF80040000835
:1071180000ED00E0002330B40568074C4B600B60BD
:107128008B600648064B012285420CBF2046184654
:1071380030BC0C31FFF7BCB8000700200044004009
:10714800FC050020014B1870704700BF4007002065
:10715800014B1878704700BF4007002070B50168E0
:10716800194A1A4B1A4C1B4E914218BF1C466368A9
:1071780004F10C05E85C00F045FD3068431C336001
:107188006368E95C144DBE29295404BF0121134AE0
:1071980003F1010308BF1170B3F5806FA8BF002386
:1071A800A5686360013DA56065B90C4C23784BB1B7
:1071B8000948FFF78BFA32682946074800F0A0F81B
:1071C8003560257070BD00BF00440040440B0020AE
:1071D800500F002014040020410700201004002054
:1071E80038B50268124B134C9A42134B134D08BF23
:1071F8001C46134B08BF1D4623680133B3F5806F47
:10720800A8BF00232360A3680133B3F5806FA36090
:1072180001DBFFF7A3FF236804F10C0101221944E5
:107228002846FFF745F80122064B1A7038BD00BF03
:1072380000440040440B0020500F0020FC050020B3
:1072480000070020400700200A4601460148FEF7D3
:10725800F5BF00BF00070020002103E00B4B5B587F
:10726800435004310A480B4B42189A42F6D30A4A53
:1072780002E0002342F8043B084B9A42F9D3FFF797
:1072880023FF00F019F8FFF7CFFA7047C0A10008F4
:1072980000000020DC030020DC0300206013002035
:1072A800FEE70A22002100F077BE0000014B1868B3
:1072B800704700BF0C02002070B500250C4E0D4C25
:1072C800A41BA410A54209D102F08AFD00250A4E8C
:1072D8000A4CA41BA410A54205D170BD56F8253050
:1072E80098470135EEE756F8253098470135F2E71B
:1072F800B8A10008B8A10008B8A10008BCA10008FE
:1073080003460244934200D1704703F8011BF9E792
:10731800002B2DE9F0471E46BBBF03F100431E4674
:1073280000232D2388B0149F129927F02007462F99
:107338001446109DDDF84CA00B7004D0452F00D1E9
:107348000135022300E0032307AA049206AA039248
:107358008DE828042246334600F082FF472F8046F6
:1073680002D1119BDB0726D5462F08EB050911D161
:1073780098F80030302B0AD10022002320463146ED
:10738800FDF776FB18B9C5F10105CAF80050DAF81F
:10739800003099440022002320463146FDF768FB5F
:1073A80038B93022079B994505D9591C07911A709D
:1073B800F8E7CDF81C904046079B159AA3EB080305
:1073C800136008B0BDE8F0870346F7B5002903F855
:1073D800022BB6BF2D222B2249420929427021DDFA
:1073E8000DF1070217460A2691FBF6F506FB151163
:1073F800092D01F1300102F8011C02F1FF34294680
:1074080009DC3031023A04F8011CBA421C4604D3A4
:10741800201A03B0F0BD2246E6E712F8011B03F874
:10742800011BF2E730221C46114404F8022B597064
:10743800EEE700002DE9F04F91B00C461A9F9346F5
:107448001E46054601F060FE036818460993FCF7DE
:10745800E7FE00230E933B680A90073323F00703E7
:1074680003F1080294F81880D4F800A03A60D3E930
:107478000023C4E91223D4F84C90A76C29F00043E8
:107488000B934FF0FF32A64B38460B99FDF722FBC2
:10749800002840F0F7814FF0FF32A14B38460B9996
:1074A800FDF7FAFA002840F0ED8100220023384663
:1074B8004946FDF7E7FA10B12D2384F84330994B7C
:1074C800994FB8F1470F98BF1F4603234FF00009A3
:1074D80023612AF00403236000965B460FAA214625
:1074E800284600F0DFF9013040F09A804FF0FF3075
:1074F80011B0BDE8F08F62680EA8531C0DF1340E70
:107508004AF4806341D1062262600021236001931E
:1075180063680DF133020590029200933A464B4698
:107528000691CDF81080CDF80CE02846FFF7F0FE64
:1075380008F0DF03472B074609D10D9BD81C02DB57
:107548006268934259DDA8F102085FFA88F8B8F139
:10755800650F0D9936D80139424604F150000D9156
:10756800FFF732FF0E9A81468318012A236102DC55
:107578002268D10701D5013323619DF83330002BF0
:10758800AAD02D2384F84330A6E7B8F1670F02D0BC
:10759800B8F1470FB9D19AB1002106910DF1330125
:1075A8008DE80C00236005903A46CDF81080CDF8A0
:1075B8000CE002914B462846FFF7AAFE0746BCE7B7
:1075C8000122A1E7B8F1660F19D1002963680CDD23
:1075D800216113B92268D20702D501330B44236114
:1075E8000D9B4FF00009A365C7E713B92268D007C0
:1075F80001D50233F3E70123F1E74FF067080D9B4C
:107608000E9A934205DB22682361D107E8D501333E
:10761800E5E7002BCCBF0123C3F102031344DEE7E7
:1076280023685A0507D423693A4659462846B0477D
:1076380001302AD15AE7B8F1650F40F2DC80D4E96D
:10764800120100220023FDF713FA002839D0012384
:10765800364A59462846B04701303FF447AF0E9B9B
:107668000D9A9A4202DB2368D8070ED50A9B099A1D
:1076780059462846B04701303FF438AF002704F197
:107688001A080E9B013B9F4211DB23689F0708D510
:10769800002704F11908E3680F9A9B1A9F42C0F269
:1076A800E780E0680F9B9842B8BF184620E701239F
:1076B800424659462846B04701303FF417AF0137D4
:1076C800DFE70D9B002B33DC0123184A5946284677
:1076D800B04701303FF40AAF0D9B23B90E9B13B995
:1076E8002368D907D1D50A9B099A59462846B04735
:1076F80001303FF4FBAE4FF0000804F11A090D9B6E
:107708005B42984501DB0E9B8EE701234A465946AA
:107718002846B04701303FF4E9AE08F10108EEE72A
:10772800FFFFEF7FF89E0008FC9E0008089F0008F6
:107738000E9AA36D9A42A8BF1A46002A904636DCD4
:107748004FF0000A04F11A0328EAE8780B93D4F8FA
:107758005890A9EB08039A4531DB0E9B0D9A9A4283
:1077680038DB2368DA0735D40E9B0D99A3EB0902A1
:10777800A3EB01089045A8BF9046B8F1000F31DC93
:10778800002728EAE87804F11A090D9A0E9B9B1A3B
:10779800A3EB08039F42BFF678AF01234A46594638
:1077A8002846B04701303FF4A1AE0137EDE7134654
:1077B80059463A462846B0470130C1D196E60123DA
:1077C8000B9A59462846B04701303FF48FAE0AF16C
:1077D800010ABCE70A9B099A59462846B047013076
:1077E800C2D183E6434607EB090259462846B0470B
:1077F8000130C5D17AE60E9A012A01DCDB0734D5BF
:1078080001233A4659462846B04701303FF46EAE48
:107818000A9B099A59462846B04701303FF466AE9C
:10782800D4E9120100220023FDF722F950B1002704
:1078380004F11A080E9B013B9F420CDB4B4604F1F6
:107848005002F2E60E9B7A1C013B59462846B04787
:107858000130F3D14AE60123424659462846B0474B
:1078680001303FF443AE0137E4E701233A46ECE741
:107878000123424659462846B04701303FF436AE08
:10788800013708E73A464B4638464946FDF722F99C
:1078980000283FF430AE014B014F12E6009F00086C
:1078A800049F00082DE9F04791461F468A680B6936
:1078B80006469342B8BF1346C9F8003091F84320F2
:1078C8000C46DDF8208012B10133C9F80030236876
:1078D800990642BFD9F800300233C9F8003025684C
:1078E80015F0060507D104F1190AE368D9F8002054
:1078F8009B1A9D422ADB94F843302268003318BF54
:10790800012392062FD404F1430239463046C0477A
:10791800013022D02368E56803F00603042B18BF62
:107928000025D9F800204FF0000908BFAD1AA36858
:10793800226908BF25EAE5759342C4BF9B1AED1872
:107948001A344D451BD10020BDE8F087012352466B
:1079580039463046C047013003D14FF0FF30BDE80B
:10796800F0870135C1E73020E11881F843005A1C3F
:1079780094F845102244023382F84310C3E70123E8
:10798800224639463046C0470130E6D009F10109A0
:10799800D7E700002DE9F04317460A7E85B06E2A26
:1079A800984606460C460C9B01F1430E00F0BC803D
:1079B8001AD8632A2ED00AD8002A00F0C880582A7C
:1079C80000F08A8004F1420584F842202AE0642A03
:1079D80001D0692AF6D121681A6811F0800F23D0E6
:1079E800111D1960136827E0732A00F0B48008D8C5
:1079F8006F2A2AD0702AE5D10A6842F020020A606C
:107A080003E0752A21D0782ADCD178226F4984F8DE
:107A1800452064E01A6801F14205111D19601368D8
:107A280084F842300123A3E011F0400F02F1040171
:107A38001960D7D0B2F90030002B03DA2D225B424F
:107A480084F8432062490A2217E02068196810F078
:107A5800800F03D0081D18600B6806E010F0400F77
:107A680001F104001860F7D00B886F2A14BF0A22AE
:107A780008225749002084F843006568002DA56056
:107A8800C0F29C80206820F004002060002B3FD1C9
:107A9800002D40F095807546082A0BD12368DA0737
:107AA80008D5236962689A42DEBF302305F8013C95
:107AB80005F1FF35AEEB05032361CDF800803B46A9
:107AC80003AA21463046FFF7EDFE013055D14FF0AD
:107AD800FF3005B0BDE8F08381F845203C492268B5
:107AE800186812F0800F00F104051D6001D00368CA
:107AF80002E05506FBD50388D00744BF42F02002B8
:107B080022601BB9226822F0200222601022B1E70D
:107B18007546B3FBF2F002FB1033CB5C05F8013D70
:107B280003460028F5D1B7E708681A6810F0800FF7
:107B3800496904D0101D18601368196007E010F037
:107B4800400F02F1040018601368F6D01980002372
:107B580075462361B1E71A68111D1960156800217F
:107B68006268284601F05CFB08B1401B60606368EE
:107B78002361002384F843309FE723692A46394666
:107B88003046C0470130A2D023689B0707D500259F
:107B980004F11909E368039A9B1A9D4205DBE06822
:107BA800039B9842B8BF184693E701234A463946D3
:107BB8003046C04701308AD00135EBE7002BA7D10A
:107BC8000B7804F1420584F8423065E71B9F0008F2
:107BD8000A9F00080FB40A4B13B51C6824B1A369A7
:107BE80013B9204601F002FA05AB049AA1682046B1
:107BF800019301F0DFFE02B0BDE8104004B0704709
:107C08000C02002038B5084B05461C6824B1A3694E
:107C180013B9204601F0EAF9A26829462046BDE8D2
:107C2800384001F0DDBF00BF0C02002070B50E46E1
:107C3800054618B183690BB901F0D8F9AB69AC688E
:107C480013B9284601F0D2F9234B9C4217D16C682E
:107C5800A3891B071DD52369DBB1013EA36816F86C
:107C6800011F013BA360E9B9002B2EDA22460A2145
:107C7800284600F0A7F9013011D00A2070BD174B33
:107C88009C4201D1AC68E3E7154B9C4208BFEC6805
:107C9800DEE72146284600F0E7F90028DDD04FF05E
:107CA800FF3070BD002B04DAA269934206DB0A2973
:107CB80004D023685A1C22601970CFE72246284650
:107CC80000F080F90130C9D1E9E70A2023685A1C7D
:107CD8002260187070BD00BF5C9F00087C9F000880
:107CE8003C9F0008024B01461868FFF79FBF00BF82
:107CF8000C02002000294FF480630CBF02220022EE
:107D080000F000B82DE9F7431D46514B04461E68A4
:107D18000F46904626B1B36913B9304601F066F9AB
:107D28004C4B9C4252D17468B8F1020F06D0B8F19E
:107D3800010F00F28980002DC0F28680214630466E
:107D480001F0EAF8616B41B104F14403994202D0B1
:107D5800304601F05DFD002363630023A361636087
:107D6800A3891B0603D52169304601F051FDA3897B
:107D7800B8F1020F23F44A6323F00303A3815DD013
:107D880001AB6A462146304601F0CCF9A389184375
:107D9800A0812DBB009D284601F028FA074600283F
:107DA8004ED1DDF80090A9453CD14FF0FF30A389B2
:107DB80043F00203A3810023A36004F14703236077
:107DC80023610123636103B0BDE8F083224B9C4229
:107DD80001D1B468A8E7214B9C4208BFF468A3E727
:107DE800002FD8D0B36913B9304601F0FFF8B8F1C5
:107DF800010F08BFA389276004BF43F00103A381D3
:107E0800A389276113F0080065611BD013F00100F6
:107E18004FF000031FBF6D42A360A561184608BF5D
:107E2800A560D0E7484601F0E1F907460028BCD034
:107E3800A3894D4643F08003A381D3E70020B6E72A
:107E4800A946F5E7A060BEE74FF0FF30BBE700BFEB
:107E58000C0200205C9F00087C9F00083C9F0008E3
:107E6800F0B5037833B1034618465E1C1B7833B966
:107E78001846F0BD0B78002B18BF0020F0BD4D1E32
:107E8800441E15F8012F002AF3D014F8017F334659
:107E98009742F6D0E8E72DE9F84F804689469246A2
:107EA8001F468B465D460A9815F8014B01F028F9E4
:107EB8002044467816F008060BD12D2C0BD101264C
:107EC8002C780BF1020567B1102F14D1302C0AD091
:107ED80011E0AB46E6E72B2C04BF2C780BF102052A
:107EE800F1E7302C27D12B7803F0DF03582B4BD147
:107EF80010276C780235002E0CBF6FF000414FF050
:107F080000410022B1FBF7FE104607FB1E1CA4F13E
:107F18003003092B11D81C46A7421DDD531C07D07E
:107F2800864516D301D1A44513DB012200FB074087
:107F380015F8014BEBE70A27DDE7A4F14103192BFC
:107F480001D8373CE8E7A4F16103192B04D8573C62
:107F5800E2E74FF0FF32EBE7531C08D12223084633
:107F6800C8F80030BAF1000F07D1BDE8F88F06B1A4
:107F78004042BAF1000F0CD022B1013DCAF80050BE
:107F8800BDE8F88F4D46F9E73024002FB3D1082714
:107F9800B1E7BDE8F88F0000084B37B51C68084DFD
:107FA800236A002B08BF2B46009313460A46014656
:107FB8002046FFF770FF03B030BD00BF0C02002061
:107FC80070020020F8B50E461446054618B18369BC
:107FD8000BB901F00BF8214B9C422AD16C68A369BC
:107FE800A360A3891A072ED5236963B32369206880
:107FF800F6B2C01A63693746984204DB2146284620
:1080080000F08AFF28BBA3680130013BA360236806
:108018005A1C22601E706369984204D0A389DB074A
:1080280019D50A2E17D12146284600F075FF90B1C0
:108038000FE00B4B9C4201D1AC68D0E7094B9C4246
:1080480008BFEC68CBE72146284600F00DF8002869
:10805800CCD04FF0FF373846F8BD00BF5C9F000812
:108068007C9F00083C9F0008324B70B51D6806468F
:108078000C4625B1AB6913B9284600F0B7FF2E4B63
:108088009C420FD16C68B4F90C309AB215072CD405
:10809800D00611D40922326043F04003A3814FF087
:1080A800FF3070BD254B9C4201D1AC68EBE7244BF7
:1080B8009C4208BFEC68E6E7510712D5616B41B1F5
:1080C80004F14403994202D0304601F0A1FB002399
:1080D8006363A38923F02403A381002363602369D6
:1080E8002360A38943F00803A38123694BB9A389BB
:1080F80003F42073B3F5007F03D02146304601F026
:1081080035F8A28912F001030CD00023A36063693B
:108118005B42A361236953B9B4F90C3013F08000B2
:10812800BAD170BD920758BF6369A360F2E7002017
:10813800F7E700BF0C0200205C9F00087C9F000846
:108148003C9F00082DE9F74F03690C6980469C4263
:1081580000F38280013C01F1140700F1140657F87E
:10816800245056F824000135B0FBF5F54FEA840E8B
:1081780006EB0E0307EB0E0901938DB34FF0000ACF
:108188003846B446D34650F8042B93B205FB03A3F4
:10819800120C4FEA134A05FB02A29BB2ABEB030396
:1081A800BCF800B04FEA124A5B441FFA82FBDCF8C5
:1081B80000208145CBEB124202EB23429BB243EAFB
:1081C80002434FEA224B4CF8043BDCD256F80E30FF
:1081D80033B9019B043B9E421A4631D3C8F810407C
:1081E800404601F03EFA002826DB30464FF0000EEC
:1081F800013557F8041BD0F800C08BB2AEEB03036F
:108208001FFA8CF213440A0CC2EB1C4202EB234205
:108218009BB243EA0243B9454FEA224E40F8043B79
:10822800E7D256F8242006EB84032AB9043B9E4281
:108238001A460BD3C8F81040284603B0BDE8F08FA3
:108248001268043B002AC9D1013CC4E71268043B08
:10825800002AEFD1013CEAE70020EEE70000000029
:108268002DE9F04F466A95B00446219DCDE90223D9
:108278003EB9102000F0BAFF606246608660066072
:10828800C660636A196851B15A68012393404A600D
:108298008B60204601F011F80022636A1A60039B84
:1082A800002BB7BF012300232B60039BAEBF2B60BD
:1082B80023F000430393DDF80C90AB4B33EA09033A
:1082C8001BD142F20F73209A1360029B23B9C9F3A2
:1082D8001300002800F08385229B53B9A34B21E0AB
:1082E800A34B06930833229A1360069815B0BDE88D
:1082F800F08F9E4B06930333F5E7DDE90267002212
:10830800002330463946FCF7B3FB804660B10123B1
:10831800209A1360229B002B00F05E85954B229AD1
:108328001360013B0693E0E712AB019313AB009394
:1083380032463B46204601F00DFAC9F30A558246FB
:10834800002D7DD03046C7F3130343F07F5141F42D
:108358004011A5F2FF35CDF840800022864BFBF78F
:108368006BFF7BA3D3E90023FCF71AF97AA3D3E9BF
:108378000023FBF763FF064628460F46FCF7AAF8DA
:1083880077A3D3E90023FCF70BF902460B463046E6
:108398003946FBF753FF06460F46FCF7B1FB0022B0
:1083A8008346002330463946FCF76CFB58B15846E3
:1083B800FCF790F802460B4630463946FCF758FB66
:1083C80008B90BF1FF3BBBF1160F58D8DDE90223C2
:1083D8006A4901EBCB01D1E90001FCF771FB0028E8
:1083E8004FD000230BF1FF3B0D93129B5D1B6B1EBF
:1083F800079343BF0023C5F1010807934FF0000816
:10840800BBF1000F3FDB079BCDF830B05B4407930F
:10841800002308931E9B092B00F2B480052BC4BFD0
:10842800043B1E931E9BC8BF0026A3F10203D8BFBE
:108438000126032B00F2B280DFE803F084862D7852
:10844800139B129D1D4405F23243202B11DD029A25
:1084580005F21240C3F1400322FA00F009FA03F3CF
:108468001843FCF727F80123A1F1F871013D109397
:1084780073E7C3F12000029B03FA00F0F1E7012340
:10848800B2E70D90B1E7CBF1000308930023A8EB06
:108498000B080C93BEE7012309931F9B002B40F3A5
:1084A80080809946049300220421656A6A6001F17C
:1084B80014029A427AD96968204600F0CAFE636AB3
:1084C80028601B68B9F10E0F069300F2F080002EA9
:1084D80000F0ED80DDE90223BBF1000FCDE90E23AA
:1084E80079DD264A0BF00F034FEA2B1602EBC30384
:1084F800F006D3E90023CDE90A235CD5DDE90E01B6
:108508001F4B0325D3E90823FCF774F9CDE90201D1
:1085180006F00F061A4F002E4FD1DDE90A23DDE9D8
:108528000201FCF767F9CDE902016EE00123099326
:108538001F9B5B4403F1010904934B46012BB8BF11
:108548000123B0E70023A7E70023F0E7AFF300809B
:1085580061436F63A787D23FB3C8608B288AC63F41
:10856800FB799F501344D33F0000F07F359F0008EC
:108578002C9F0008099F00080000F83FD09F0008C2
:10858800A89F00080126002309961E934FF0FF3389
:1085980000220493994612231F9284E7012309932A
:1085A800F4E70123049399461A46F5E76A684900F7
:1085B80001326A607BE70225ACE7F10708D5DDE9FF
:1085C8000A01D7E90023FBF7EBFFCDE90A010135E2
:1085D800761008379FE700F0A580DDE90E01CBF1A2
:1085E8000006A24B06F00F0203EBC203D3E90023F7
:1085F800FBF7D6FF02250023CDE902019C4F361177
:10860800002E40F08480002B8DD10D9B002B00F0B4
:108618008B80DDE90223CDE90A23DDE90A01002286
:10862800944BFCF72FFA00287ED0B9F1000F7BD0CD
:10863800049B002B37DDDDE90A0100228E4BFBF796
:10864800AFFFCDE90201049E0BF1FF370135284643
:10865800FBF740FFDDE90223FBF7A2FF874B00226F
:10866800FBF7ECFDCDE90A010B9BA3F150750B95C7
:10867800002E5CD1DDE902010022814BFBF7DCFD15
:108688000A9A2B46CDE90201FCF71AFA002840F0B5
:10869800F782DDE902010A9A05F10043FCF7F2F9D5
:1086A800002840F0EB82DDE90E23CDE90223139B7D
:1086B800002BC0F25081BBF10E0F00F34C816B4BC5
:1086C80003EBCB03D3E90023CDE904231F9B002B45
:1086D80080F2DA80B9F1000F00F3D68040F0CD8245
:1086E800DDE904010022664BFBF75AFFDDE90223AE
:1086F800FCF7DCF94E464F46002840F0A482069B62
:10870800069A5D1C31230BF1010B13709FE2F207EF
:1087180005D5D7E90023FBF743FF01230135761080
:1087280008376DE7022570E75F464E468FE7069AE1
:108738004E4B32441192099A711E002A48D003EB1D
:10874800C103D3E9002300204E49FCF753F8DDE9C3
:108758000A23FBF771FDCDE90A01069DDDE9020157
:10876800FCF7CEF90646FBF7B5FE02460B46DDE9F7
:108778000201FBF761FDDDE90A23303605F8016BDC
:10878800CDE90201FCF77EF9002864D1DDE9022376
:1087980000203849FBF750FDDDE90A23FCF772F9A0
:1087A800002840F0B980119B9D423FF47CAFDDE981
:1087B8000A010022304BFBF7F3FE0022CDE90A0143
:1087C800DDE902012C4BFBF7EBFECDE90201C5E721
:1087D80003EBC101D1E90001DDE90A23FBF7E0FE63
:1087E800CDE90A01069DDDE90201FCF789F9064693
:1087F800FBF770FE02460B46DDE90201FBF71CFDA4
:108808003036119B05F8016BAB42CDE902014FF000
:10881800000224D11B4BDDE90A01FBF70FFD0246DC
:108828000B46DDE90201FCF74BF9002874D1DDE9BC
:108838000A2300201349FBF7FFFC02460B46DDE93B
:108848000201FCF71FF900283FF42DAF15F8013C91
:108858006A1E302B01D0BB464DE01546F6E7064BA5
:10886800FBF79EFECDE90201BDE700BFD09F0008DF
:10887800A89F00080000F03F0000244000001C40B2
:10888800000014400000E03F069DDDE90267DDE9D5
:10889800042330463946FBF7ADFFFCF731F9804633
:1088A800FBF718FEDDE90423FBF77AFE02460B46C8
:1088B80030463946FBF7C0FC08F1300605F8016B75
:1088C800069E0246AE1BB1450B4637D1FBF7B6FCF8
:1088D80006460F4602460B46DDE90401FCF7D2F8CE
:1088E800C8B9DDE9040132463B46FCF7C1F810B1CE
:1088F80018F0010F0FD15146204600F0DEFC00238E
:10890800209A2B700BF101031360229B002B3FF47C
:10891800ECAC1D60E9E45F4615F8012C6B1E392AA2
:1089280006D1069A9A4207D13023137013460137AD
:108938001A7801321A708EE71D46EDE70022B54B12
:10894800FBF72EFE0022002306460F46FCF790F8A0
:1089580000289CD0CFE7099A002A00F029811E9AA6
:10896800012A00F30E81109A002A00F0068103F212
:1089780033434546089E079A01211A4420469844E5
:10898800079200F03AFD0746002D0BDD079B002BF0
:1089980008DDAB42A8BF2B46079AA8EB0308ED1ADF
:1089A800D31A0793089BFBB1099B002B00F00481A5
:1089B800002E11DD39463246204600F0B3FD5246FE
:1089C80001460746204600F021FD51460A90204600
:1089D80000F073FC0A9B9A46089B9A1B04D05146E8
:1089E800204600F09FFD82460121204600F005FD4B
:1089F8000C9B0646002B40F3E1801A4601462046B0
:108A080000F090FD1E9B0646012B40F3DA80002300
:108A18000893336906EB8303186900F0A0FCC0F1E2
:108A28002000079B184410F01F0000F0F080C0F1F0
:108A38002003042B40F3E280079BC0F11C00804414
:108A4800054403440793B8F1000F05DD514642463B
:108A5800204600F0B5FD8246079B002B05DD314618
:108A68001A46204600F0ACFD06460D9B002B00F090
:108A7800D3803146504600F0F4FD002880F2CC80C7
:108A8800002351460A22204600F02EFC099B0BF1D8
:108A9800FF3B8246002B00F0A981002339460A22B9
:108AA800204600F021FC049B0746002B03DC1E9B9C
:108AB800022B00F3B980002D05DD39462A462046F1
:108AC80000F07EFD0746089B002B00F010817968B6
:108AD800204600F0BEFB05463A6907F10C01023258
:108AE80092000C3000F0AAFB01222946204600F033
:108AF80067FD07970746029BDDF8188003F001031E
:108B0800089331465046FFF71DFB0799054600F1CB
:108B18003009504600F0A5FD3A46029031462046FD
:108B280000F0B9FDC3680246002B40F0E280014620
:108B38000990504600F095FD0346099A11462046D3
:108B4800099300F0BAFB099B002B40F0D4801E9AD1
:108B5800002A40F0D080089A002A40F0CC80B9F171
:108B6800390F00F0E880029B002B01DD05F1310987
:108B780008F1010588F800906BE0129BC3F13603F9
:108B8800F7E6089B09F1FF36B342B7BF089B9E1B67
:108B9800F21A0C9BBFBF08969B180C930026B9F1DC
:108BA800000FB9BFA8EB0905002345464B46E2E68E
:108BB800089E4546099FE7E6089A10E71E9B012B89
:108BC80018DC029BB3B9039BC3F31303A3B9039B3C
:108BD80023F000431B0D1B052BB1079B08F101086F
:108BE80001330793012308930C9B002B7FF411AFEB
:108BF800012016E70023F6E7029BF4E73FF423AFD2
:108C0800079A1C331A4498441D4413461AE703462E
:108C1800F6E700BF00002440B9F1000F33DC1E9BCB
:108C2800022B30DDCDF81090049B63B93146052244
:108C3800204600F059FB01460646504600F011FD5B
:108C480000283FF75CAD1F9B069D6FEA030B0023CE
:108C580007933146204600F030FB002F3FF44BAE1F
:108C6800079B2BB1BB4203D01946204600F025FBD9
:108C78003946204600F021FB3DE600263746E2E76C
:108C8800BB4637463BE5099BCDF81090002B7FF497
:108C980012AF069D31465046FFF754FA069B00F185
:108CA800300905F8019B049AEB1A9A4200F3818077
:108CB800069B012AACBF9B180133984600230793F3
:108CC80051460122204600F07BFC3146824600F0E6
:108CD800C8FC002834DC02D119F0010F30D1454618
:108CE80015F8013C6A1E302BB3D11546F8E7384613
:108CF800FFE6012322E7029A002A04DB28D11E9A04
:108D080032BB089A22BB002B7FF732AF51460122B3
:108D1800204600F055FC3146824600F0A2FC0028AF
:108D280005DC7FF425AF19F0010F3FF421AFB9F14D
:108D3800390F7FF41BAF392308F1010808F8013C0B
:108D4800454615F8013C6A1E392B3AD001333FE0FD
:108D5800002B08F1010505DDB9F1390FEBD009F158
:108D6800010907E7069B049AEB1A9342A84605F8FF
:108D7800019CA5D0514600230A22204600F0B4FAEF
:108D8800079B8246BB424FF00A024FF00003079947
:108D9800204604D100F0A8FA07900746B1E600F093
:108DA800A3FA002307900A223946204600F09CFACD
:108DB800F3E7514600230A22204600F095FA82463E
:108DC80068E7069B934205D13123069A0BF1010B04
:108DD80013703EE71546B4E7094BFFF7A3BA229B89
:108DE800002B7FF47DAA074BFFF79CBA049B002B4E
:108DF8003FF74FAF1E9B022B7FF74BAF14E700BF27
:108E0800089F00082C9F00088A892DE9F041054633
:108E180010070C465AD44B68002B05DC0B6C002B52
:108E280002DC0020BDE8F081E66A002EF9D00023BC
:108E380012F480522F682B6033D0606DA3895A07D3
:108E480005D56368C01A636B0BB1236CC01A002385
:108E58000246E66A216A2846B047431CA38906D120
:108E680029681D294BD82B4ACA40D60747D5002266
:108E780062602269D904226004D5421C01D12B68A2
:108E880003B96065616B2F600029CAD004F14403FF
:108E9800994202D0284600F0BBFC00206063BDE880
:108EA800F081216A01232846B047411CC6D12B68AE
:108EB800002BC3D01D2B01D0162B01D12F60B0E79A
:108EC800A38943F04003A381BDE8F0810F69002F17
:108ED800A7D0930718BF00230E6808BF4B69A6EBFD
:108EE80007080F608B60B8F1000F9ADD43463A46D9
:108EF800216A2846A66AB047002807DCA38943F000
:108F08004003A3814FF0FF30BDE8F0810744A8EB90
:108F18000008E8E70100402038B50B6905460C4613
:108F2800DBB118B183690BB900F060F80C4B9C42B7
:108F380009D16C68B4F90C307BB121462846BDE8EC
:108F48003840FFF761BF074B9C4201D1AC68F1E79D
:108F5800054B9C4208BFEC68ECE7002038BD00BF19
:108F68005C9F00087C9F00083C9F0008014900F0B6
:108F7800A9B800BF218F0008002310B5044603607C
:108F88004360836081814366C28103614361836179
:108F9800194608225C30FEF7B3F9054B2462636278
:108FA800044BA362044BE362044B236310BD00BF70
:108FB800759C0008979C0008CF9C0008F39C00084B
:108FC80070B568254A1E55430E4605F1740100F038
:108FD8006BFC044640B1002180E842000C30A060E0
:108FE80005F16802FEF78CF9204670BD836910B55B
:108FF800044633BB8364C3640365124B124A1B687F
:109008008262984204BF0123836100F01FF8606008
:10901800204600F01BF8A060204600F017F8002258
:10902800E06004216068FFF7A7FF01220921A0681A
:10903800FFF7A2FF02221221E068FFF79DFF01233C
:10904800A36110BDF49E0008758F0008F8B51C4B8D
:1090580007461E68B36913B93046FFF7C7FF48369D
:10906800B4687368013B03D5336833B13668F7E7F2
:10907800B4F90C506DB16834F4E704213846FFF7B1
:109088009FFF30600028F1D10C2304463B60204646
:10909800F8BD4FF6FF73E38101236566A381256060
:1090A800A560656025616561A5610822294604F10E
:1090B8005C00FEF725F96563A563A564E564E6E74A
:1090C800F49E00082DE9F84380468946002600F101
:1090D800480414B93046BDE8F883A5686768013FBD
:1090E80001D52468F5E7AB89012B07D9B5F90E300E
:1090F800013303D029464046C84706436835EEE7A2
:10910800D0F8EC0070470000044B1B68186A044B49
:10911800002808BF1846F030704700BF0C02002036
:109128007002002070B50E46B1F90E1090B00029FB
:1091380014461D4607DA00232B60B3891A0610D49B
:109148004FF480630EE001AA00F002FE0028F2DB73
:10915800029A02F47042A2F500535A425A412A6018
:10916800EEE740230020236010B070BD8B8973B5F3
:109178009D0706460C4607D504F147032360236183
:109188000123636102B070BD01AB6A46FFF7CAFFF5
:1091980000990546304600F087FB48B9B4F90C3011
:1091A8009A05EFD423F0030343F00203A381E3E716
:1091B8000D4BB362A389206043F08003A381009B19
:1091C80020616361019B5BB1B4F90E10304600F079
:1091D800D1FD28B1A38923F0030343F00103A38140
:1091E800A3891D43A581CDE7758F0008024B014671
:1091F800186800F059BB00BF0C02002082B001B90A
:1092080001A942B14BB113780B601278101C18BF3A
:10921800012002B070471046FBE76FF00100F8E745
:1092280010B5C9B202449042034601D1002010BDD6
:109238001C7801308C42F6D1184610BD10B5431E7B
:109248000A44914200D110BD11F8014B03F8014FB7
:10925800F7E770B5456A04460E463DB91020FFF79A
:10926800C5FF6062456085600560C560656AEB683A
:1092780083B1636ADB6853F82600B8B9012101FAA3
:1092880006F56A1D9200204600F0B3FA60B1466008
:1092980085600EE021220421204600F0AAFA636AC4
:1092A800E860DB68002BE4D1002070BD026843F859
:1092B800262000230361C36070BD70B5446A06466A
:1092C8000D463CB91020FFF791FF7062446084603E
:1092D8000460C4603DB1736A6A68DB6853F82210A1
:1092E800296043F8225070BD2DE9F0411F4606461B
:1092F8000C4600230D6901F1140EDEF8000001335D
:1093080081B202FB0171000C0F0C02FB007089B2E4
:1093180001EB00419D424FEA10474EF8041BECDC7C
:10932800D7B1A3689D4212DB616830460131FFF76F
:1093380090FF8046226904F10C01023292000C3041
:10934800FFF77CFF21463046FFF7B7FF444604EBA2
:10935800850301355F6125612046BDE8F081020C77
:1093680012040346B2B90304102013F07F4F04BF60
:109378001B02083013F0704F04BF1B01043013F0B8
:10938800404F04BF9B000230002B06DB5B0003D577
:10939800013070470020E8E7202070470368014645
:1093A80013F007020BD0DA0723D4980749BF5B08EC
:1093B8009B0801200B605CBF0B600220704798B2CD
:1093C800A8B910201B0C13F0FF0F04BF1B0A0830AC
:1093D8001A0704BF1B0904309A0704BF9B08023010
:1093E800DA0702D45B0806D001300B6070471046DC
:1093F800E9E7002070472020704710B50C4601218E
:10940800FFF727FF01224461026110BD2DE9F74FE4
:1094180014460A69236989469A42BEBF0B46A1468B
:109428001C46D9F81070D4F810A0D9F80830D9F82B
:10943800041007EB0A069E42C8BF0131FFF709FF77
:1094480000F114052B46002205EB8608434516D388
:1094580004F1140209F1140102EB8A0301EB8707F6
:109468000193019C134694420CD8002E03DD58F852
:10947800043D002B54D0066103B0BDE8F08F43F8DB
:10948800042BE3E7B3F800A00432BAF1000F20D0B0
:10949800AE4689464FF0000C59F8044BBEF800B0B0
:1094A800A3B20AFB03B34FEA144BDEF8004063444F
:1094B8004FEA144C0AFB0BC404EB13449BB243EA77
:1094C80004434F454FEA144C4EF8043BE4D8CEF819
:1094D80000C032F8029CB9F1000F1FD0AE468C468E
:1094E8004FF0000A2B68BCF80040BEF802B09BB2EF
:1094F80009FB04B4A24443EA0A434EF8043B5CF86F
:10950800043BBEF800401B0C09FB0343674503EB13
:109518001A434FEA134AE6D8CEF800300435A0E7DC
:10952800013EA2E72DE9F843154612F0030206466C
:109538000F4607D0214C013A002354F82220FFF7A8
:10954800D3FE0746AD1035D0746A3CB91020FFF73A
:109558004DFE7062446084600460C460D6F8248064
:10956800D8F808404CB940F271213046FFF745FF62
:1095780000230446C8F8080003604FF00008EB0712
:109588000AD5394622463046FFF740FF814639461C
:109598003046FFF792FE4F466D100BD0206838B961
:1095A800224621463046FFF731FF2060C0F8008090
:1095B8000446E4E73846BDE8F88300BF98A00008F1
:1095C8002DE9F0470C460746164623694FEA621A0A
:1095D8000AEB03094968A36809F10105AB4231DBCD
:1095E8003846FFF736FE00228046114600F1140384
:1095F80052452ADB20692AEAEA7A04F1140116F0B6
:109608001F0203EB8A0301EB800E22D00020C2F177
:10961800200C0E689640304343F8040B51F8040BB5
:109628008E4520FA0CF0F4D8186008B109F102054B
:10963800013D3846C8F810502146FFF73EFE404627
:10964800BDE8F08701315B00C8E743F8221001321A
:10965800CEE7043B51F8042B8E4543F8042FF9D884
:10966800E6E703690A6930B59B1A0CD192001430F9
:1096780014318418114454F8045D51F8042D9542AE
:1096880003D005D30123184630BDA042F3D3FAE72F
:109698004FF0FF33F7E72DE9F0470D46074611462F
:1096A80028461446FFF7DDFF061E08D13146384626
:1096B800FFF7CFFD012346610361BDE8F087A4BF32
:1096C80023462C4638466168A6BF1D46002601265B
:1096D800FFF7BFFD4FF0000CC6602B69266904F147
:1096E800140205F1140902EB860709EB830800F15F
:1096F800140152F804AB59F8045B1FFA8AF3634467
:10970800ACB21B1B2C0CC4EB1A4404EB23449BB2D5
:109718004FEA244CC84543EA0444964641F8044BB2
:10972800E7D8BE4505D351F8043D8BB10661BDE8C5
:10973800F0875EF8044BA2B26244131403EB14439F
:1097480092B242EA03424FEA234C41F8042BE8E77D
:10975800013EE8E72DE9F3411C4601219046089EA9
:10976800099DFFF776FDC4F31302C4F30A540746B4
:1097780034BB0192B8F1000F27D002A840F8088D39
:10978800FFF70CFE0099F0B1019AC0F1200302FA2C
:1097980003F30B43C2407B610192019B002B14BF72
:1097A80002210121BB613961C4B1A4F233440444EC
:1097B8003460C0F135002860384602B0BDE8F08159
:1097C80042F48012D5E77961E7E701A8FFF7E6FDE3
:1097D8000121019B39617B612030E5E7A0F232402D
:1097E80007EB810330601869FFF7B9FDC0EB411042
:1097F800E1E738B502FB01F4214600F055F80546CB
:1098080018B122460021FDF77BFD284638BD00002F
:1098180038B50546002943D051F8043C0C1F002BED
:10982800B8BFE41800F0C8FA1E4A1368104633B9E6
:10983800636014602846BDE8384000F0BEBAA34211
:109848000BD921686218934201BF1A685B685218E5
:10985800226063600460EDE713465A680AB1A242C9
:10986800FAD919685818A0420BD120680144581831
:1098780082421960DED110685268014419605A604A
:10988800D8E702D90C232B60D4E7206821188A4234
:1098980001BF116852680918216062605C60C9E7FD
:1098A80038BD00BF1804002070B5CD1C25F0030595
:1098B80008350C2D38BF0C25002D064601DBA942C2
:1098C80003D90C233360002070BD00F075FA234AD9
:1098D8001468214691B9224C23681BB9304600F020
:1098E800B5F920602946304600F0B0F9431C26D16E
:1098F8000C233046336000F060FAE4E70B685B1B2A
:109908001AD40B2B0FD90B60CC18CD50304600F071
:1099180054FA04F10B00231D20F00700C31A1BD0D2
:109928005A42E25070BD8C420BBF63684B681360AB
:10993800636018BF0C46E9E70C464968CAE7C41CCF
:1099480024F00304A04205D0211A304600F07EF925
:109958000130CDD02560D9E770BD00BF18040020C4
:109968001C040020936810B4013B002B936008DAB4
:109978009469A34202DBCBB20A2B02D110BCFEF7DA
:1099880021BB1368581C10601970C8B210BC70470E
:10999800F8B506460F461446D518AC4201D100204A
:1099A80007E03A4614F8011B3046FFF7DBFF431C7B
:1099B800F3D1F8BD2DE9F04F9DB00C46174603933F
:1099C800064618B183690BB9FFF710FB7C4B9C4224
:1099D80057D17468A38918075DD52369002B5AD01D
:1099E8000023099320238DF8293030234FF0010BF1
:1099F8008DF82A30B846454615F8013B002B55D15D
:109A0800B8EB070A0BD053463A4621463046FFF7D3
:109A1800BFFF013000F0C480099B5344099398F8B4
:109A28000030002B00F0BC8000234FF0FF3204937D
:109A38000793059206938DF853301A9305222978D7
:109A48006048FFF7EDFB05F10108049B002831D1C0
:109A5800D90644BF20228DF853201A0744BF2B2271
:109A68008DF853202A782A2A2CD000210A20079A18
:109A7800A84698F800300135303B092B6DD971B3F1
:109A880026E0514B9C4201D1B468A3E74F4B9C425E
:109A980008BFF4689EE721463046FEF7E5FA00283D
:109AA8009ED04FF0FF301DB0BDE8F08F252BA7D01A
:109AB800A846A0E7434A4546801A0BFA00F0184327
:109AC8000490BBE7039A111D12680391002A01DB79
:109AD800079204E0524243F002030792049398F875
:109AE80000302E2B10D198F8013008F101012A2BF3
:109AF80037D1039B08F102081A1D1B680392002B3B
:109B0800B8BF4FF0FF330593314D032298F800108A
:109B18002846FFF785FB40B14023401B03FA00F0BD
:109B2800049B08F101080343049398F800100622E7
:109B3800284808F101078DF82810FFF771FB002865
:109B480034D0254B03BB039B073323F007030833AB
:109B58000393099B4B4409934CE700FB0232012114
:109B680086E700230A2518460593884698F80020BA
:109B78000131303A092A03D9002BC5D00590C3E733
:109B880005FB00200123F0E703AB00932246134BAB
:109B980004A93046FDF74EFCB0F1FF3F8146D8D10D
:109BA800A3895B063FF57DAF09987CE703AB00937B
:109BB80022460A4B04A93046FDF7ECFEECE700BF4D
:109BC8005C9F0008A4A000087C9F00083C9F000838
:109BD800AAA00008AEA000083D74000899990008E2
:109BE80070B50D461446064618B183690BB9FFF7E0
:109BF800FDF9134B9C4212D17468A368013B002BFA
:109C0800A36016DAA269934202DBEBB20A2B10D1E9
:109C1800224629463046BDE87040FEF7D3B9094BC5
:109C28009C4201D1B468E8E7074B9C4208BFF4683E
:109C3800E3E72368E8B25A1C22601D7070BD00BFBC
:109C48005C9F00087C9F00083C9F000838B50023F3
:109C5800054C054608462360FDF710FA431C02D15F
:109C6800236803B12B6038BD5C13002010B50C4687
:109C7800B1F90E1000F0A2F80028ABBF636DA389FC
:109C88001B1823F48053ACBF6365A38110BD2DE975
:109C9800F0411F468B890546DB050C46164605D55F
:109CA80002230022B1F90E1000F074F8A38932469D
:109CB80023F48053A381B4F90E103B462846BDE82F
:109CC800F04100F023B810B50C46B1F90E1000F0C1
:109CD80061F8431CA38915BF606523F4805343F4DE
:109CE8008053A38118BFA38110BDB1F90E1000F0F5
:109CF8001FB849B1FF2A8BBF8A230A70036001206D
:109D080088BF4FF0FF3070470846704738B50546A2
:109D1800084611460022054C22601A46FCF744FD0D
:109D2800431C02D1236803B12B6038BD5C130020AB
:109D380038B50023054C054608462360FDF7B8F9F9
:109D4800431C02D1236803B12B6038BD5C1300208B
:109D580038B50023064C0546084611462360FDF732
:109D6800AAF9431C02D1236803B12B6038BD00BF98
:109D78005C13002038B50023054C054608462360CF
:109D8800FDF79EF9431C02D1236803B12B6038BD4F
:109D98005C13002038B50546084611460022054CDC
:109DA80022601A46FDF78EF9431C02D1236803B1DD
:109DB8002B6038BD5C1300207047704738B50546E6
:109DC800084611460022054C22601A46FDF748F95C
:109DD800431C02D1236803B12B6038BD5C130020FB
:109DE800F8B500BFF8BC08BC9E467047F8B500BF80
:089DF800F8BC08BC9E46704750
:109E000002030405060708090A0B0C0D0E0F1010BB
:109E1000000102030405060708090A41542B4357B1
:109E20004D4F44453D330D0A0041542B4349504D9D
:109E300055583D310D0A0041542B43575341503D75
:109E400022424C55455F54455354222C22222C3536
:109E50002C300D0A0041542B43495053455256456E
:109E6000523D312C343030300D0A0041542B4349DF
:109E70004653520D0A004553502053657474696E61
:109E80006720436F6D706C657465200D002B495021
:109E9000442C302C33303A000D0A202564205265C2
:109EA00073756C74203A2000256420004920616D90
:109EB000206E6F7420666F756E640D00556172744C
:109EC000205374617274200D004372632067656EC5
:109ED0006572617465202578200D0A00000000007D
:109EE000000000000102030406070809000000004A
:109EF0000102030410020020494E4600696E66000C
:109F00004E414E006E616E003000303132333435D8
:109F100036373839414243444546003031323334D4
:109F2000353637383961626364656600496E666943
:109F30006E697479004E614E000000000000000060
:109F40000000000000000000000000000000000011
:109F50000000000000000000000000000000000001
:109F600000000000000000000000000000000000F1
:109F700000000000000000000000000000000000E1
:109F800000000000000000000000000000000000D1
:109F90000000000000000000000000004300504FDF
:109FA000534958002E0000000080E03779C3414338
:109FB000176E05B5B5B89346F5F93FE9034F384D2F
:109FC000321D30F94877825A3CBF737FDD4F1575DB
:109FD000000000000000F03F0000000000002440EE
:109FE00000000000000059400000000000408F40C9
:109FF000000000000088C34000000000006AF84034
:10A000000000000080842E4100000000D012634157
:10A010000000000084D797410000000065CDCD41CD
:10A02000000000205FA00242000000E876483742AE
:10A03000000000A2941A6D42000040E59C30A2424C
:10A040000000901EC4BCD64200003426F56B0C43C1
:10A050000080E03779C3414300A0D8855734764368
:10A0600000C84E676DC1AB43003D9160E458E143C9
:10A07000408CB5781DAF154450EFE2D6E41A4B443E
:10A0800092D54D06CFF08044F64AE1C7022DB54483
:10A09000B49DD9794378EA44050000001900000016
:10A0A0007D000000232D302B2000686C4C0065667D
:10A0B000674546470000202020202020202020281F
:10A0C0002828282820202020202020202020202070
:10A0D00020202020202088101010101010101010A8
:10A0E00010101010101004040404040404040404E8
:10A0F0001010101010101041414141414101010167
:10A10000010101010101010101010101010101013F
:10A11000011010101010104242424242420202024C
:10A12000020202020202020202020202020202020F
:10A1300002101010102000000000000000000000BD
:10A14000000000000000000000000000000000000F
:10A1500000000000000000000000000000000000FF
:10A1600000000000000000000000000000000000EF
:10A1700000000000000000000000000000000000DF
:10A1800000000000000000000000000000000000CF
:10A1900000000000000000000000000000000000BF
:10A1A00000000000000000000000000000000000AF
:08A1B0000000000000000000A7
:04A1B8000D4200084C
:04A1BC00E94100086D
:10A1C0000100000010000000000021104220633058
:10A1D0008440A550C660E770088129914AA16BB1FF
:10A1E0008CC1ADD1CEE1EFF13112100273325222A7
:10A1F000B5529442F772D662399318837BB35AA34F
:10A20000BDD39CC3FFF3DEE3622443342004011476
:10A21000E664C774A44485546AA54BB5288509959E
:10A22000EEE5CFF5ACC58DD5533672261116300646
:10A23000D776F6669556B4465BB77AA719973887EE
:10A24000DFF7FEE79DD7BCC7C448E5588668A77806
:10A250004008611802282338CCC9EDD98EE9AFF93E
:10A26000488969990AA92BB9F55AD44AB77A966AE6
:10A27000711A500A333A122AFDDBDCCBBFFB9EEB8E
:10A28000799B588B3BBB1AABA66C877CE44CC55CB6
:10A29000222C033C600C411CAEED8FFDECCDCDDDDE
:10A2A0002AAD0BBD688D499D977EB66ED55EF44E86
:10A2B000133E322E511E700E9FFFBEEFDDDFFCCF2E
:10A2C0001BBF3AAF599F788F8891A981CAB1EBA182
:10A2D0000CD12DC14EF16FE18010A100C230E320FE
:10A2E0000450254046706760B9839893FBA3DAB3A6
:10A2F0003DC31CD37FE35EF3B1029012F322D2324E
:10A300003542145277625672EAB5CBA5A895898575
:10A310006EF54FE52CD50DC5E234C324A01481049D
:10A320006674476424540544DBA7FAB79987B89745
:10A330005FE77EF71DC73CD7D326F2369106B016ED
:10A3400057667676154634564CD96DC90EF92FE905
:10A35000C899E9898AB9ABA944586548067827683D
:10A36000C018E1088238A3287DCB5CDB3FEB1EFBE5
:10A37000F98BD89BBBAB9ABB754A545A376A167A8D
:10A38000F10AD01AB32A923A2EFD0FED6CDD4DCDB5
:10A39000AABD8BADE89DC98D267C076C645C454CDD
:10A3A000A23C832CE01CC10C1FEF3EFF5DCF7CDF85
:10A3B0009BAFBABFD98FF89F176E367E554E745E2D
:10A3C000932EB23ED10EF01E0024F40010020020A5
:10A3D000000000005C9F00087C9F00083C9F000874
:10A3E000000000000000000000000000000000006D
:10A3F000000000000000000000000000000000005D
:10A40000000000000000000000000000000000004C
:10A41000000000000000000000000000000000003C
:10A42000000000000000000000000000000000002C
:10A4300043000000000000000000000000000000D9
:10A44000000000000000000000000000000000000C
:10A4500043000000000000000000000000000000B9
:10A4600000000000000000000000000000000000EC
:10A470004300000000000000000000000000000099
:10A4800000000000000000000000000000000000CC
:10A490004300000000000000000000000000000079
:10A4A00000000000000000000000000000000000AC
:10A4B0004300000000000000000000000000000059
:10A4C000000000000000000000000000000000008C
:10A4D0004300000000000000000000000000000039
:10A4E000000000000000000000000000000000006C
:10A4F0004300000000000000000000000000000019
:10A50000000000000000000000000000000000004B
:10A51000FB9C00080592000800000000B5A00008A0
:10A52000A49F0008DB9E0008DB9E0008DB9E00085D
:10A53000DB9E0008DB9E0008DB9E0008DB9E000817
:10A54000DB9E0008DB9E0008FFFFFFFFFFFFFFFF11
:10A55000FFFFFFFFFFFF0000010041534349490097
:10A5600000000000000000000000000000000000EB
:10A570000000000000000000000041534349490072
:10A5800000000000000000000000000000000000CB
:0CA59000000000000000000000000000BF
:04000005080072611C
:00000001FF
